:020000040000FA
:10000000F42A8A0121088207463400347634003409
:1000100053340034633400343E34003484340034C8
:1000200053340034633400344634003476340034BE
:100030005334003463340034343400343A340134FB
:10004000343400349D340034533400346334003489
:1000500046340034EB340034463400347634003413
:1000600053340034633400343E3400348434003478
:10007000533400346334003446340034763400346E
:10008000533400346334003446340034EB340034E9
:1000900046340034763400344A3400346F3400344B
:1000A0004F340034D234003437340034283401342F
:1000B00037340034283401343E34003408340134F9
:1000C0003E34003484340034423400347D3400340F
:1000D00046340034D63401344634003476340034A7
:1000E0004A3400346F3400344F340034A3340134C4
:1000F0004F340034693400345334003463340034F2
:10010000693400343A3401344634003476340034EF
:1001100053340034633400343E34003484340034C7
:1001200053340034633400344634003476340034BD
:100130005334003463340034343400343A340134FA
:10014000343400349D340034533400346334003488
:1001500046340034EB3400348A01210882074634E7
:1001600000347634003453340034633400343E3485
:10017000003484340034533400346334003446345F
:10018000003476340034533400346334003446345D
:100190000034EB34003446340034763400344A34CE
:1001A00000346F3400344F340034D23400343734E8
:1001B00000342834013437340034283401343E34D8
:1001C0000034083401343E34003484340034423482
:1001D00000347D34003446340034D63401343734AE
:1001E0000034943400343E340034843400345334C6
:0E01F000003463340034463400347634003476
:1002000001308A00210882074F34003469340034F9
:100210005E34003458340034693400349D34003482
:10022000693400349D3400340234003444341634CC
:1002300001308A002108820753340034C634003468
:10024000343400343A34013437340034283401343F
:100250003E34003484340034423400347D3400347D
:100260003E34003484340034533400346334003476
:100270003E34003484340034463400347634003460
:100280004F34003469340034533400346334003460
:100290004F3400346934003446340034763400344A
:1002A0003E340034843400344F3400346934003434
:1002B000533400345134023453340034C6340034DF
:1002C0004F340034D234003453340034C634003454
:1002D000423400347D340034533400346334003409
:1002E00037340034943400344634003476340034E7
:1002F0002E3400346034013453340034C6340034B6
:100300004F340034D234003453340034C634003413
:100310003E340034843400345334003463340034C5
:10032000343400349D3400343E340034843400349A
:10033000293400348C34013453340034C63400344E
:10034000343400343A34013437340034283401343E
:100350003E34003484340034423400347D3400347C
:100360003E34003484340034533400346334003475
:100370003E3400348434003446340034763400345F
:100380004F3400346934003453340034633400345F
:100390004F34003469340034463400347634003449
:1003A0003E340034843400344F3400346934003433
:1003B000533400345134023453340034C6340034DE
:1003C0004F340034D234003453340034C634003453
:1003D000423400347D340034533400346334003408
:1003E00037340034943400344634003476340034E6
:0803F0002E34003460340134A6
:1004000002308A00210882074F34003469340034F6
:100410005334003463340034583400345D340034D1
:100420005334003463340034343400349D340034A5
:1004300037340034943400343E340034083401340A
:100440003E34003408340134023400344434163469
:1004500002308A00210882074F3400343B340134D3
:1004600053340034633400345E3400345834003480
:10047000693400344E3400344F340034A334013432
:100480003E340034083401343434003474340234DB
:100490002E3400346034013446340034C134023424
:1004A0003B340034A43401343E340034843400340A
:1004B00046340034763400344F3400346934003428
:1004C00053340034293401344F3400346934003457
:1004D0005E34003458340034533400346334003410
:1004E00069340034EC34003446340034763400345B
:1004F0003E340034843400343B3400348C340034D3
:100500003734003451340234343400343A34013452
:100510004F3400343B3401345334003463340034FA
:100520005E34003458340034693400344E340034BE
:100530004F340034A33401343E34003408340134E1
:100540002C340034EC3402342E3400346034013462
:100550003B3400343034023446340034EB3400345D
:1005600046340034763400344A3400346F34003476
:1005700046340034763400343E340034843400345D
:100580003B3400348C3400342E340034B034003426
:1005900034340034D73401344F34003469340034F7
:1005A00046340034763400344F3400346934003437
:1005B0005334003429340134343400349D3400344D
:1005C0003B3400348C340034463400347634003408
:1005D0004F340034D23400344F340034D234003439
:1005E000023400344434163483161F308500FE3044
:1005F0008600831207231A232D2307231A232D2372
:100600004023532307231A232D23662363002A3014
:10061000A000A1010120A200A10A0120A300A10ABB
:100620000120A400A10A0120A500A10A7923A00BA2
:100630000A2B08001430A000A101AC20A200A10ADE
:10064000AC20A300A10AAC20A400A10AAC20A50004
:10065000A10A7923A00B1D2B08000530A000A101E1
:100660000021A200A10A0021A300A10A0021A400E8
:10067000A10A0021A500A10A7923A00B302B0800B4
:100680003830A000A1011821A200A10A1821A3005E
:10069000A10A1821A400A10A1821A500A10A792302
:1006A000A00B432B08000930A000A1010022A200EA
:1006B000A10A0022A300A10A0022A400A10A00228C
:1006C000A500A10A7923A00B562B08003230A00008
:1006D000A1012822A200A10A2822A300A10A2822FF
:1006E000A400A10A2822A500A10A7923A00B692B46
:1006F00008002308A7002203A600260A0319A7035F
:1007000006142208A8002308A9009523061026082D
:10071000A8002708A9009523A403240A0319A50308
:1007200024082504031D802B0800A803280A0319A8
:0C073000A90328082904031D952B0800CC
:02400E00103D63
:00000001FF
